:10001600F894EE27ECBBE8E1E1BDE0E1E1BDEE27B7
:10002600E5BF80E890E0A0E6BB27ED930197E9F7EE
:10003600E8E4F5E0C895102C3196C89531966E2FF8
:100046007F2FF02DE12D3097A1F0C895A02D319688
:10005600C895B02D3196C895802D3196C895902DAE
:100066003196C8950D9231960197D9F7E62FF72F5D
:10007600E1CFEFEDF0E0EDBFFEBFCFE7D0E044C249
:10008600219774D2EE2309F003C0EE272196089536
:10009600E981EE2309F419C0E5E5EA93ADD221968C
:1000A600EE27E883E981EF5FE983E150AE2FBB27B6
:1000B600EC91EA93A1D22196E881EF5FE883AE2F17
:1000C600A83008F001C0EECF04C0ECECEA9394D25D
:1000D6002196E1E0219608952297EA81EA93D0DFFE
:1000E6002196EE2309F003C0EE2722960895EEEB43
:1000F600EA9382D22196EE27E983E0E8E883E88155
:10010600EF5FE883E150EF9372D2AF91BB27EC9398
:10011600E981EF5FE983AE2FA93008F001C0EFCF88
:10012600E0E8EA93E9E0EA9371D222969ED222961B
:100136000895E881EA93A4DF2196EE2309F003C02F
:10014600E1EFF8ED0895E4E4EA9356D22196E6E26B
:10015600F2E0FA93EA93FFD12296E881EA93BCDFB4
:100166002196EE2309F003C0E1EFF8ED0895FED1E4
:10017600A1E8BB27EC91FF27E7FDFFEFFE2FEE2757
:10018600FF93EF93A0E8BB27EC91AF91BF91FF27B8
:10019600EA2BFB2BA5E0B0E06DD20895EA81EA9345
:1001A6006FDF2196EE2309F002C0EE270895EEE4F4
:1001B600EA9322D22196E881EA931ED22196E9811A
:1001C600EA931AD22196EA81EA9386DF2196EE23F4
:1001D60009F002C0EE270895A3E8BB27EC91AE2FE5
:1001E600E981EA1709F009C0A2E8BB27EC91AE2F16
:1001F600E881EA1709F001C002C0EE270895EA81F6
:10020600EA933EDF2196EE2309F002C0EE27089519
:10021600E8E4EA93F1D12196EFE0FF27FA93EA9317
:100226009AD12296A3D10895A1000A003F06DBCFFA
:10023600666D7D077F6FE0919400F0919500309791
:100246000CF03FC0AFE8E0E4BB27EC93ACE8E9E391
:10025600BB27EC93E0919400F0919500FA93EA9312
:1002660072D12296E0939400F0939500EDE8EF9317
:10027600A0919400B0919500EAE0F0E02ED2A1EAB8
:10028600AE0FBB27EC91AF91BB27EC93EEE8EF9353
:10029600A0919400B0919500EAE0F0E002D2A1EAC4
:1002A600AE0FBB27EC91AF91BB27EC93AEE8BB2713
:1002B600EC91EF3309F004C0AEE8EE27BB27EC93D0
:1002C60053C0ACE8E9E3BB27EC93EFE8EF93A091CA
:1002D6009400B0919500E4E6F0E0E3D1A1EAAE0F18
:1002E600BB27EC91AF91BB27EC93A0919400B09102
:1002F6009500E4E6F0E0F1D1E0939200F0939300EC
:10030600EDE8EF93A0919200B0919300EAE0F0E05F
:10031600E4D1A1EAAE0FBB27EC91AF91BB27EC93DA
:10032600EEE8EF93A0919200B0919300EAE0F0E03E
:10033600B8D1A1EAAE0FBB27EC91AF91BB27EC93E6
:10034600AFE8BB27EC91EF3309F00EC0AFE8EE271C
:10035600BB27EC93AEE8BB27EC91EF3309F004C062
:10036600AEE8EE27BB27EC930895E0919C00F09150
:100376009D00E0939E00F0939F00E0919A00F0911B
:100386009B00E0939C00F0939D00E0919800F09113
:100396009900E0939A00F0939B00E0919600F0910B
:1003A6009700E0939800F0939900E0919400F09103
:1003B6009500E0939600F0939700E0919800F091F5
:1003C6009900A0919600B0919700EA0FFB1FA091AB
:1003D6009A00B0919B00EA0FFB1FA0919C00B09180
:1003E6009D00EA0FFB1FA0919E00B0919F00AE0FEB
:1003F600BF1FE5E0F0E055D1E0939400F09395003F
:100406000895E0919000F09191003196E09390006C
:10041600F0939100AE2FBF2FE5E0F0E0AE17BF07D7
:1004260008F416C0EE27E0939000E0939100EFEFFA
:10043600E8BBEE27EA937DDE2196AE2FBF2FEAE0DA
:10044600F0E02FD1E0939400F09395008EDFF3DE79
:1004560008950F921F926F937F938F939F93AF93FD
:10046600BF93CF93DF93EF93FF930FB60F92E09175
:100476008900EF5FE093890005C0EE27E0938900CD
:10048600C0DF05C0FF27D7D080040F0000000F9003
:100496000FBEFF91EF91DF91CF91BF91AF919F91E9
:1004A6008F917F916F911F900F9018952197E0E2A1
:1004B600E0938B00EFEFE093A000EE27E883A8819E
:1004C600A4300CF01FC005C0E881EF5FE883E1505F
:1004D600F6CFE0918B00E095E2BBE881ACE8AE0F89
:1004E600BB27EC91E095E8BBE1E0FF27FA93EA939E
:1004F60032D02296EFEFE8BBE0918B00E695E093D1
:100506008B00E2CF21960895EFEFE7BBEE27E8BB1D
:10051600EFE7E1BBEE27E2BBE5E0E3BFEE27E2BF94
:10052600E2E0E9BFE0E8E8B921D078941FD0E2E242
:10053600FF27E0939400F09395007DDEB7DFFECFB2
:1005460008952E020000E881F98130971AF4E095AB
:10055600F09531960895E881F981309631F088EE6C
:1005660093E00197F1F73197D1F70895EE27969822
:100576008E9A80EE91E00197F1F78E9883E18A9545
:10058600F1F7869B089585E68A95F1F7869BE395B4
:1005960086E891E00197F1F708958E9A83E08A95AF
:1005A600F1F78E988FE08A95F1F7889486990894EA
:1005B600E7958BE68A95F1F70895E8948E9A83E09D
:1005C6008A95F1F770FD8E9881E18A95F1F7869903
:1005D60003C070FF03C0089570FF089584E68A95EE
:1005E600F1F78E9887E08A95F1F76894089568E0A8
:1005F600D4DF6A95E9F7089568E07881EE27DDDFB4
:1006060026F477956A95D9F7E3950895EE278881BC
:10061600882381F068E1A981BA8198E0FD917F2F56
:100626007E27779508F4E627E795F6959A95B9F724
:100636008A9599F70895AE2FBF2FFF91EF91EE0F90
:10064600FF1FC8953196802DC8953196902D00963E
:1006560049F0C8953196A015C8951190B00589F74F
:10066600E82FF92FF695E7950994EE23E1E009F0D6
:10067600EE27089536D005D01EF4E095F095319614
:1006860008950A2E1B2E81E1AA27BB1B05C010F474
:10069600A00DB11DB695A795F795E7958A95B9F77B
:1006A60008951FD005D01EF4E095F0953196089573
:1006B6000024112490E1AA0FBB1F001C111C0E1A66
:1006C6001F0A18F40E0E1F1E01C0A1609A9599F715
:1006D600EA2FFB2FA02DB12D0895E3DFEA2FFB2F84
:1006E6000895E894F7FF04C0E095F0953196689474
:1006F600B7FF06C0A095B095119600F8039400FACE
:02070600089554
:100000000AC0FECFFDCFFCCFFBCFFACF25C2F8CF81
:06001000F7CFF6CFF5CF9B
:00000001FF
